:107800000C94283C0C94433C0C94433C0C94433C17
:107810000C94433C0C94433C0C94433C0C94433CEC
:107820000C94433C0C94433C0C94433C0C94433CDC
:107830000C94433C0C94433C0C94433C0C94433CCC
:107840000C94433C0C94433C0C94433C0C94433CBC
:1078500011241FBECFE5D8E0DEBFCDBF10E0A0E60B
:10786000B0E0E6E5FFE702C005900D92A036B10753
:10787000D9F711E0A0E6B0E001C01D92A43AB1072B
:10788000E1F70C94703F0C94003C0F93EF93FF933F
:107890003ED0FC01062F35D0FF91EF910F91089556
:1078A0000F930F921F92EF93FF9331D0FC010B01C6
:1078B00001E027D0FF91EF911F900F900F91089555
:1078C0000F930F92EF93FF9322D0FC0160FD67BFEF
:1078D000C895802DE395C895902DFF91EF910F905D
:1078E0000F9108950F930F9212D0082E09E009D03E
:1078F0000F900F9108950F930AD001E102D00F91DC
:107900000895E199FECF07BFE895FFFF000007B794
:1079100000FDFDCF089583E089B9549A539A0895E4
:107920008CB19927089540E050E04817590750F46A
:107930002AE633E000002150304037FFFBCF4F5F95
:107940005F4FF3CF08958BB1992780789070089599
:107950005498539808950E94A83C0C9400000895F0
:107960008CB95E9BFECF5E9A08950E94A33C88234B
:10797000E1F30E94903C803219F481E090E0089598
:1079800085E10E94B03C80E090E008950895EF9278
:10799000FF920F931F93CF93DF937B01C0E0D0E062
:1079A000C617D70770F48C010E94A33C8823E1F32B
:1079B0000E94903CF80181938F012196CE15DF053E
:1079C00098F381E090E0DF91CF911F910F91FF90AC
:1079D000EF90089590E0282F33272138310589F062
:1079E0002238310524F42038310549F00DC0223801
:1079F000310549F02839310539F493E005C092E0AA
:107A000003C091E001C092E1892F9927089540E0D9
:107A100050E06091A0007091A10046175707E8F46C
:107A2000E2EAF0E08091A2018EBB8091A2019091E8
:107A3000A301292F33272FBB01969093A301809395
:107A4000A20180818DBBE29AE19AE199FECF4F5F5E
:107A50005F4F31964617570728F308950F931F93EA
:107A6000CF93DF9300E010E08091A0009091A100FF
:107A700008171907D8F4C2EAD0E08091A2019091CA
:107A8000A301880F991F60E0800F911F0E94603C46
:107A90008883892F992789830E5F1F4F22968091B3
:107AA000A0009091A1000817190738F3DF91CF913A
:107AB0001F910F9108958091A0009091A1000097CF
:107AC000C1F0E2EAF0E0AC018091A2018EBB8091AE
:107AD000A2019091A301292F33272FBB01969093E8
:107AE000A3018093A201E09A8DB38193415050404D
:107AF00059F708950F931F93CF93DF938C0161156E
:107B0000710541F0EB01F80181918F010E94B03CB9
:107B10002197C9F781E090E0DF91CF911F910F91FC
:107B20000895EF92FF920F931F93CF93DF93C0E0DE
:107B3000D0E08E017E01CFE7D0E0F092A301E09289
:107B4000A20163E0C8010E94453C219780E490E0D7
:107B5000E80EF91E00581F4FD7FFEFCF0E947B3C65
:107B6000DF91CF911F910F91FF90EF900895EF92C9
:107B7000FF920F931F93CF93DF9300E010E080916B
:107B8000A0009091A1000817190708F047C0EE2443
:107B9000FF24E801CD55DF4FF801EE55FF4FEE0D04
:107BA000FF1D4081888122969927382F2227240F94
:107BB000311D8091A2019091A301880F991FB901F5
:107BC0008E0D9F1D0E94503C82E090E0E80EF91E51
:107BD00090E8E916F10400F38091A2019091A301CD
:107BE000880F991F63E0800F911F0E94453C809190
:107BF000A2019091A301880F991F65E0800F911F4A
:107C00000E94453C0E947B3C00581F4F8091A00081
:107C10009091A1000817190708F4B9CFDF91CF910F
:107C20001F910F91FF90EF900895CF93C0E069E00E
:107C300081E090E00E94603C84FF03C08F7E0E9440
:107C4000723C0E94A33C8823E1F30E94903C992758
:107C500082359105DCF4803591050CF054C08134F7
:107C6000910509F45AC0823491053CF480339105A2
:107C700009F449C0C19759F12FC18234910509F423
:107C80005FC08534910509F45EC026C18635910533
:107C900009F4EDC0873591054CF48235910509F45E
:107CA00061C08535910509F465C016C18437910519
:107CB00009F4A0C0853791052CF48436910509F4A8
:107CC00072C00AC18537910509F4C1C005C10E947F
:107CD000B53C882309F4B5CF84E10E94B03C81E42F
:107CE0000E94B03C86E50E94B03C82E50E94B03C18
:107CF00080E20E94B03C83E50E94B03C84E50E9493
:107D0000B03C8BE406C00E94B53C882309F499CFAF
:107D100084E10E94B03C80E1E0C061E070E080E678
:107D200090E00E94C73C0E94B53C882309F489CFAB
:107D300084E10E94B03C809160000E94EA3CE9CF5F
:107D400064E170E00AC061E070E080E690E00E94CB
:107D5000C73C809160009927BC0180E690E00E94BA
:107D6000C73CD1CF0E94B53C882309F46ACF0E945A
:107D7000913DCECF62E070E080E690E00E94C73C8B
:107D80000E94B53C882309F45CCF2091600080916B
:107D900061009927982F8827820F911D9093A30146
:107DA0008093A201B5CF63E070E080E690E00E948E
:107DB000C73C20916100809160009927982F882707
:107DC000820F911D9093A1008093A000BC0182EAD4
:107DD00090E00E94C73C0E94B53C882309F431CF53
:107DE00080916200863419F40E94B73D91CF0E94C1
:107DF000073D8ECF63E070E080E690E00E94C73CD4
:107E000020916100809160009927982F8827820F28
:107E1000911D9093A1008093A0000E94B53C8823FF
:107E200009F40FCF80916200863419F40E942E3D30
:107E300002C00E945B3D84E10E94B03C6091A000C2
:107E40007091A10082EA90E00E947A3D64CF0E9486
:107E5000B53C882309F4F5CE84E10E94B03C8EE164
:107E60000E94B03C85E90E94B03C81E052CF64E0C2
:107E700070E080E690E00E94C73C0E94B53C8823F9
:107E800009F4DFCE84E10E94B03C8091600080352F
:107E900031F480916100882361F4C82F17C08835C0
:107EA00031F480916100883061F4C3E00FC0803507
:107EB00031F480916100883049F4C2E007C0883510
:107EC00029F480916100882309F4C1E069E08C2FD6
:107ED00099270E94603C1DCF85E10E94B03CB1CE45
:107EE000CFE5D8E0DEBFCDBFCEE1F8948EEF93E0D2
:107EF0000E94A23F843B59F48FEF93E00E94A23F7F
:107F0000833C29F48DEF93E00E94A23F81BF0E9441
:107F10008B3C0E94903C84E690E00E94933C0E943F
:107F2000A33C882321F4C150C8BBCC23A1F7CC23A8
:107F300019F00E94153E02C00E94AB3C80E090E028
:107F40000C94AA3FE199FECF9FBB8EBBE09A992784
:067F50008DB30895FFCF80
:040000030000780081
:00000001FF
